:100000000C946B000C9493000C9493000C9459097D
:100010000C9459090C9459090C9493000C94930076
:100020000C9493000C9493000C9493000C94930004
:100030000C9493000C9493000C9493000C949300F4
:100040000C94A21A0C9493000C94961D0C94C81D49
:100050000C9493000C9493000C9493000C949300D4
:100060000C9493000C94930000000008000201001F
:100070000003040700000000000000000102040863
:100080001020408001020408102001020408102002
:10009000040404040404040402020202020203032E
:1000A00003030303000000002300260029000000D2
:1000B0000000250028002B0000000000240027007D
:1000C0002A0035082C0B391061146F147A14571656
:1000D0006216F81DA61E11241FBECFEFD8E0DEBFAA
:1000E000CDBF12E0A0E0B1E0E8ECF1E502C0059080
:1000F0000D92A03BB107D9F724E0A0EBB2E001C01C
:100100001D92A430B207E1F710E0C6EDD0E004C0C4
:100110002297FE010E94FD23C23CD107C9F70E942D
:10012000B61E0C94E2280C9400000F931F93CF93FB
:10013000DF938C018FE190E00E94C51EEC0120E06E
:1001400046E067E00E94250AF801D183C08340E8B9
:1001500055E260E070E0CE01DF91CF911F910F91E9
:100160000C94550AEF92FF920F931F93CF93DF9356
:1001700000D000D000D0CDB7DEB78C017B0164E1A8
:1001800071E0CE0101960E94B120B701CE01019627
:100190000E940D22BC01F801828193810E94201FE0
:1001A000CE0101960E944320F801808191810E9436
:1001B0003009B701F801808191810E94201F2696A5
:1001C0000FB6F894DEBF0FBECDBFDF91CF911F9168
:1001D0000F91FF90EF900895FC01808191810C9424
:1001E000D51FCF93DF93EC01FB01608171810E94E9
:1001F000DB1FCE01DF91CF910895AF92BF92CF92D6
:10020000DF92EF92FF920F931F93CF93DF93CDB7BF
:10021000DEB762970FB6F894DEBF0FBECDBF7C018C
:1002200061E08AE00E94B91B61E08AE00E94F21B53
:100230006AE171E0F701808191810E94321F69E2D9
:1002400071E0F701808191810E94321F89E093E083
:10025000F701938382835701F4E0AF0EB11CB5011F
:100260000E9403139E01295F3F4F6901892B59F5B5
:1002700066E371E0F701808191810E94321F00E006
:1002800020E04FEF6FEFCE0101960E947F1E01E04C
:1002900020E04EEF69EAC6010E947F1E01EB21E0DB
:1002A0004EEF69EACE010D960E947F1E8E010F5F10
:1002B0001F4F9601AE01435F5F4FB501F701828189
:1002C00093810E94C91369E571E0F70180819181F2
:1002D0000E94131F69E073E0CE0101960E943E1454
:1002E0008E010D5F1F4FF80161918F014AE050E0D0
:1002F000F701808191810E94A01F64E871E0F701FD
:10030000808191810E94131F0C151D0561F7F70173
:10031000808191810E941C1F62960FB6F894DEBF07
:100320000FBECDBFDF91CF911F910F91FF90EF9046
:10033000DF90CF90BF90AF90089526E0EEE0F1E01F
:10034000DC01149601900D922A95E1F7FC0171836E
:1003500060830C94FD000F931F93CF93DF938C0168
:100360008FE190E00E94C51EEC0120E048E069E0CA
:100370000E94250AF801D183C08340E855E260E07D
:1003800070E0CE01DF91CF911F910F910C94550A2F
:10039000CF93DF93EC0162EA72E002960E94B120F3
:1003A000CE01DF91CF910C94AB01EF92FF920F93AE
:1003B0001F93CF93DF9300D000D000D0CDB7DEB72E
:1003C0008C01DC018D919C910E943009F8018081A3
:1003D0009181DC01ED91FC910480F581E02D09957E
:1003E000892B79F0F801819191917F01DC01ED91E8
:1003F000FC910680F781E02D0995682FC7010E94C6
:10040000FA21F801868197810E97B8F00E5F1F4F91
:100410002DE030E041E050E0B801CE0101960E94AD
:10042000A922BE016F5F7F4FC8010E941D21CE012E
:1004300001960E94432081E001C080E026960FB61D
:10044000F894DEBF0FBECDBFDF91CF911F910F910A
:10045000FF90EF90089560E771E002960E942022DD
:1004600091E0811101C090E0892F089562EA72E065
:1004700002960C94292162E082E00E94B91B62E09E
:1004800083E00C94B91BCF93C62F82E00E94281CF6
:10049000892B11F4C13049F483E00E94281C892B78
:1004A00031F481E0C23021F402C081E001C080E07B
:1004B000CF91089582E00E94281C892B11F481E0DD
:1004C000089582E00895EF92FF920F931F93CF93C8
:1004D000DF93CDB7DEB72C970FB6F894DEBF0FBE13
:1004E000CDBF8C016DE771E0FC01808191810E949C
:1004F000321F84E090E00E94C51E7C01F8018081DB
:100500009181F70193838283C7010E949500F801CE
:10051000F382E2828AE090E00E94C51E7C01F8012D
:10052000608171810E949D01F801F582E48288E07A
:1005300090E00E94C51E7C010E94C801F801F7826C
:10054000E68281E090E00E94C51E7C010E943B0291
:10055000F801F186E0860E94111AAB01BC012AE085
:10056000CE0107960E949A2166E871E0CE010196BD
:100570000E94B120BE01695F7F4FCE0101960E94AB
:100580000D22BC01F801808191810E94201FCE01C3
:1005900001960E944320CE0107960E9443202C968C
:1005A0000FB6F894DEBF0FBECDBFDF91CF911F9184
:1005B0000F91FF90EF900895CF92DF92EF92FF920C
:1005C0000F931F93CF93DF93EC017B018FEF8A870B
:1005D0008B878C871D868E01025F1F4F6E018EE315
:1005E000C80ED11C62EA72E0C8010E94B1200A5F05
:1005F0001F4F0C151D05B1F762EA72E0C8010E9499
:10060000B120F982E882CE01DF91CF911F910F9145
:10061000FF90EF90DF90CF900C9463028F929F92A7
:10062000AF92BF92CF92DF92EF92FF920F931F9300
:10063000CF93DF93CDB7DEB7A1970FB6F894DEBFA7
:100640000FBECDBF8C016B017A0169E871E0C60174
:100650000E942022882309F4BFC020E030E04EE051
:1006600050E0BE016F5F7F4FC7010E943F2240E113
:1006700050E060E070E0CE0101960E944F26AB0191
:10068000BC012AE0CE0146960E946D216DE871E022
:10069000CE0140960E94B120BE016A5E7F4FCE011E
:1006A00040960E940D22BC01CE014C960E9414215E
:1006B000CE0140960E944320CE0146960E944320E0
:1006C0000E94111AAB01BC012AE0CE0146960E949D
:1006D0009A2162E971E0CE0140960E94B120BE01EC
:1006E0006A5E7F4FCE0140960E940D22BC01CE0172
:1006F0004C960E94F321CE0140960E944320CE01E9
:1007000046960E944320F8016385772767FD709520
:100710004AE0CE0146960E94412169E971E0CE018E
:1007200040960E94B120BE016A5E7F4FCE01409686
:100730000E940D22BC01CE014C960E94F321CE01F5
:1007400040960E944320CE0146960E944320F80125
:100750006485772767FD70954AE0CE0146960E9432
:1007600041216FE971E0CE0140960E94B120BE01A7
:100770006A5E7F4FCE0140960E940D22BC01CE01E1
:100780004C960E94F321CE0140960E944320CE0158
:1007900046960E944320C8010E94E505BE01645EA2
:1007A0007F4F882331F0F801808191810E94201FC2
:1007B00010C0CE0140960E941421BE01605F7F4FA1
:1007C000F801828193810E94B200CE0140960E947E
:1007D0004320CE014C9660C068EA71E0C6010E94D9
:1007E0002022882319F06AE971E009C06CEA71E0FF
:1007F000C6010E942022882309F160EA71E0CE013F
:1008000040960E94B120B701CE0140960E940D2271
:10081000BC01CE0101960E941421BE016F5F7F4F83
:10082000F801828193810E94B200CE0101960E945C
:100830004320CE0140960E944320EAC063EB71E062
:10084000C6010E942022882351F1C7010E944D2336
:100850000E94E0190E94111AAB01BC012AE0CE01EE
:1008600040960E949A2166E871E0CE0101960E94AE
:10087000B120BE01605F7F4FCE0101960E940D2224
:10088000BC01F801808191810E94201FCE01019658
:100890000E944320CE0140960E944320B9C068EBDD
:1008A00071E0C6010E942022882331F0C7010E9416
:1008B0004D23F8016387ACC06FEB71E0C6010E9465
:1008C0002022882331F0C7010E944D23F80164875C
:1008D0009FC069EC71E0C6010E942022882321F0AC
:1008E00081E0F801858794C06EEC71E0C6010E943A
:1008F0002022882331F0C7010E944D23F80162872E
:1009000087C067ED71E0C6010E942022882309F4A8
:1009100058C05801FEE0AF0EB11CC12CD12C6CE7C1
:10092000C7010E94852296012F5F3F4F4901019622
:1009300069F426E02C9DC0012D9D900D11240E968A
:10094000B701800F911F0E94FD2038C06CE7C701DE
:100950000E9485229C0140E050E0B701CE01019643
:100960000E94A922BE016F5F7F4FC5010E941D2119
:10097000CE0101960E9443206CE7C7010E948522A8
:10098000F70124813581AC014F5F5F4FB701CE0184
:1009900001960E94A922BE016F5F7F4FC7010E948E
:1009A0001D21CE0101960E9443206401F6E0AF0EA6
:1009B000B11C28E08216910409F0B1CFF8018286BB
:1009C00027C061EE71E0C6010E942022882301F158
:1009D000F80182851816E4F46801FEE0CF0ED11C00
:1009E000E12CF12CF8018285992787FD9095E81676
:1009F000F9066CF4B601F801808191810E94201FF4
:100A0000FFEFEF1AFF0A26E0C20ED11CEBCF1286D1
:100A1000A1960FB6F894DEBF0FBECDBFDF91CF9188
:100A20001F910F91FF90EF90DF90CF90BF90AF900C
:100A30009F908F900895CF92DF92EF92FF920F9345
:100A40001F93CF93DF93CDB7DEB768970FB6F894B7
:100A5000DEBF0FBECDBF7C018B016AEE71E0CE011F
:100A600001960E94B120B801CE0101960E940D228C
:100A7000BC01F701808191810E94201FCE01019667
:100A80000E944320C8010E94EE2262EA72E0CE0179
:100A900043960E94B12062EA72E0CE010D960E9458
:100AA000B1206DE971E0CE0101960E94B120BE0136
:100AB0006F5F7F4FC8010E94A5226C01CE01019695
:100AC0000E944320CD20C09409F468C06DE971E014
:100AD000CE0107960E94B120BE01695F7F4FC80119
:100AE0000E94A5229C0140E050E0B801CE01019691
:100AF0000E94A922BE016F5F7F4FCE0143960E94E4
:100B00001D21CE0101960E944320CE0107960E942E
:100B100043206DE971E0CE0107960E94B120BE012D
:100B2000695F7F4FC8010E94A522F80124813581A9
:100B3000AC014F5F5F4FB801CE0101960E94A92220
:100B4000BE016F5F7F4FCE010D960E941D21CE0129
:100B500001960E944320CE0107960E944320BE01C9
:100B6000635F7F4FCE0101960E941421BE016D5E2E
:100B70007F4FCE0107960E941421AE014F5F5F4F59
:100B8000BE01695F7F4FC7010E940E03CE01079629
:100B90000E944320CE0101960E944320CE010D9673
:100BA0000E944320CE0143960E94432068960FB6D0
:100BB000F894DEBF0FBECDBFDF91CF911F910F9193
:100BC000FF90EF90DF90CF9008950F931F93CF93F6
:100BD000DF93CDB7DEB72C970FB6F894DEBF0FBE0C
:100BE000CDBF8C0148EE53E060E070E0FC018081F5
:100BF00091810E94D51FF801158660EF71E0808118
:100C000091810E94321FF801608171814AE0CE011A
:100C100007960E94DB1F62EA72E0CE0107960E94EF
:100C20002022811111C0BE01695F7F4FCE01019664
:100C30000E941421BE016F5F7F4FC8010E941B05F7
:100C4000CE0101960E944320F8011585CE0107963A
:100C50000E944320812F2C960FB6F894DEBF0FBE62
:100C6000CDBFDF91CF911F910F910895EF92FF9229
:100C70000F931F93CF93DF93CDB7DEB72C970FB6AB
:100C8000F894DEBF0FBECDBF8C01DC0116968D91AE
:100C90009C9117970E94D501882309F45DC0F80143
:100CA000868197810E942B02882309F450C081E03D
:100CB000D8011C969C91913009F480E0F80184875A
:100CC000668177816E5F7F4FCE0107960E94142167
:100CD00069E871E0CE0101960E94B120AE01495F42
:100CE0005F4FBE016F5F7F4FC8010E940E03CE01B0
:100CF00001960E944320CE0107960E944320D8010E
:100D00001C966C91772767FD70954AE0CE01079697
:100D10000E9441216CEA71E0CE0101960E94B1204F
:100D2000AE01495F5F4FBE016F5F7F4FC8010E94F8
:100D30000E03CE0101960E944320CE0107960E9429
:100D4000432068EE73E080E090E00E941B1BF801F6
:100D5000868197810E943602D8018D919C91DC0199
:100D6000ED91FC910480F581E02D0995892B41F1ED
:100D7000F80180819181DC01ED91FC910680F78181
:100D8000E02D0995F801FE967F018A30A9F4BF0194
:100D9000CE0101960E941421BE016F5F7F4FC801F2
:100DA0000E941B05CE0101960E94432062EA72E078
:100DB000C7010E94292104C0682FCF010E94FA2197
:100DC000D8011B966C911B9718968D919C91199741
:100DD0000E944302882369F1F801808591850E9471
:100DE0005A02D8011B968C93682F772767FD709560
:100DF0004AE0CE0107960E94412168EA71E0CE01E7
:100E000001960E94B120AE01495F5F4FBE016F5F46
:100E10007F4FC8010E940E03CE0101960E9443201D
:100E2000CE0107960E944320F801868197810E9497
:100E300036022C960FB6F894DEBF0FBECDBFDF9101
:100E4000CF911F910F91FF90EF9008950F931F93F3
:100E5000CF93DF93CDB7DEB72C970FB6F894DEBFF4
:100E60000FBECDBF8C0148EE53E060E070E0FC01A6
:100E7000828193810E94EC006EEF71E0CE010196B9
:100E80000E94B120BE016F5F7F4FF8018281938184
:100E90000E94B200CE0101960E944320F8016281B7
:100EA00073814AE0CE0101960E94F100BE016F5F9E
:100EB0007F4FC8010E941B05CE0101960E9443206E
:100EC00067E072E0CE0101960E94B120BE016F5F23
:100ED0007F4FF801828193810E94B200CE0101967A
:100EE0000E944320F801628173814AE0CE0101969D
:100EF0000E94F100BE016F5F7F4FC8010E941B0579
:100F0000CE0101960E944320C8010E94E505882376
:100F100009F44CC063E172E0CE0101960E94B12059
:100F2000BE016F5F7F4FF801828193810E94B20002
:100F3000CE0101960E944320F801628173814AE04C
:100F4000CE0101960E94F100BE016F5F7F4FC80184
:100F50000E941B05CE0101960E944320F801828564
:100F6000181624F563E272E0CE0101960E94B120CA
:100F7000BE016F5F7F4FF801828193810E94B200B2
:100F8000CE0101960E944320F801628173814AE0FC
:100F9000CE0101960E94F100BE016F5F7F4FC80134
:100FA0000E941B05CE0101960E944320C8010E94A9
:100FB000E5058823E9F060E372E0CE0101960E9426
:100FC000B12061EE71E0CE0107960E94B120AE0122
:100FD0004F5F5F4FBE01695F7F4FC8010E940E03E4
:100FE000CE0107960E944320CE0101960E94432025
:100FF0002C960FB6F894DEBF0FBECDBFDF91CF9118
:101000001F910F910895CF93DF9326E040E855E2BA
:1010100060E070E08BE593E00E94341D84E490E092
:101020000E94C51EEC016BE573E00E94DC02D093C8
:10103000B102C093B00262E372E08BE593E00E94DC
:10104000321F8091B0029091B1020E94260760E4A5
:1010500072E08BE593E0DF91CF910C94321F809189
:10106000B0029091B1020C9436060F9300E020E09C
:1010700040E060E082EB92E00E947F1E0F910895B5
:10108000CF93CFB7F8948091B802811127C0EAE9D5
:10109000F0E08491E6E8F0E09491E82FF0E0EE0FC4
:1010A000FF1FE854FF4FA591B4918C91892321F43F
:1010B00061E08AE00E94F21B61E08AE00E94B91BB5
:1010C0008CB580618CBD8CB580648CBD61E08DE099
:1010D0000E94B91B61E08BE00E94B91B8091B802AD
:1010E0008F5F8093B802CFBFCF9108952091FB020C
:1010F0003091FC0228173907B9F49091B902809118
:10110000BA02981789F0E091B902F0E0E554FD4F7A
:1011100080812091B90230E02F5F3F4F2F7333273A
:101120002093B90290E008958FEF9FEF08951F93E9
:10113000CF93DF93DC015C968D919C915D97009736
:1011400049F481E090E013969C938E93129780E08F
:1011500090E03BC05196ED91FC91529750962C91A6
:101160005097322F30951FB75E964C915E9741FB9A
:10117000772770F941FD6095F8944081772311F04D
:10118000422B01C043234083EC012197F1F748E053
:10119000508160FF02C0522B01C053235083EC01E9
:1011A0002197F1F76695415099F78081772311F0E7
:1011B000832301C0822B80831FBF5C968D919C91FD
:1011C0005D970197F1F781E090E0DF91CF911F915A
:1011D000089508952091FB023091FC0228173907E9
:1011E00071F49091B9028091BA02981741F0E091A0
:1011F000B902F0E0E554FD4F808190E008958FEF53
:101200009FEF08952091FB023091FC0228173907C7
:1012100071F48091BA022091B90290E0805C9F4FF6
:10122000821B910960E470E00E946923089580E0C8
:1012300090E00895E091FB02F091FC02E817F907B5
:1012400069F4A389B4899C918589809589238C93BD
:101250001092FC021092FB0281E0089580E0089554
:10126000CF93DF93EC018A8D9B8D892BF1F08091D8
:10127000FB029091FC028C179D07B9F0009711F0CA
:101280000E941A098E8D8E7F8E8F1092BA02109254
:10129000B902D093FC02C093FB02EB89FC898081E8
:1012A0009D89892B808381E001C080E0DF91CF910F
:1012B00008951F920F920FB60F9211242F933F9310
:1012C0004F935F936F937F938F939F93AF93BF934E
:1012D000EF93FF93E091FB02F091FC02309709F449
:1012E00051C0868DA685B785958581FF04C08C91F8
:1012F000892329F447C08C91892309F043C0A3892D
:10130000B4899C918589809589238C938689978956
:101310000197F1F7208D318DA685B785758558E049
:1013200040E0C9010197F1F7842F90E095958795EA
:10133000482F6C91672309F04068515091F7868DD2
:1013400081FD40958091BA0290E001968F739927B4
:101350002091B902281749F0A091BA02B0E0A55433
:10136000BD4F4C938093BA0203C0868D8160868FF7
:10137000828D938D0197F1F7A389B4898C9195891A
:10138000892B8C93FF91EF91BF91AF919F918F919A
:101390007F916F915F914F913F912F910F900FBE71
:1013A0000F901F9018951F93CF93DF93EC01162F8A
:1013B0006E8D6695617081E06827812F0E94F21B17
:1013C00061E0812F0E94B91B812F90E0FC01E4585D
:1013D000FF4FE491E88BFC01E057FF4FE491F0E010
:1013E000EE0FFF1FE255FF4F859194919A8B898BE9
:1013F000DF91CF911F9108951F93CF93DF93EC015D
:10140000162F60E0812F0E94B91B8E8D81FD04C0D4
:1014100061E0812F0E94F21B1C87812F90E0FC016C
:10142000E458FF4FE491ED87FC01E057FF4FE49152
:10143000F0E0EE0FFF1FEC55FF4F859194919F87D1
:101440008E87DF91CF911F910895FF920F931F9385
:10145000CF93DF93EC01F62E522F1B821A8208EEF7
:1014600013E020E030E00C831D832E833F8383E56F
:1014700092E0998388831F8A1E8A198E188E1B8E8C
:101480001A8E1D8E1C8E8E8D8E7F50FB81F98E8F55
:10149000642FCE010E94D3096F2DCE01DF91CF9131
:1014A0001F910F91FF900C94FC09CF93DF93EC01F7
:1014B0009A01AB011B8E1A8E198E188E1F8A1E8AF6
:1014C00060E079E08DE390E00E949F23C901243021
:1014D000310520F0B9016350710902C061E070E08C
:1014E0007D8F6C8FEC85E63108F068C0B901769588
:1014F00067956431710518F06351710902C061E0AC
:1015000070E07F8B6E8B069718F0C901059702C0BB
:1015100081E090E0998F888FC901880F991F820F11
:10152000931F96958795969587958D30910510F028
:101530000C9702C081E090E09B8F8A8F2091680019
:10154000E83050F091E0EE3008F490E081E001C026
:10155000880F9A95EAF701C084E0822B8093680097
:101560002C85283038F02E3040F0263148F48CE6B7
:1015700090E008C08DE690E005C08BE690E002C0E8
:1015800080E090E09C8B8B8B283030F481E001C0B0
:10159000880F2A95EAF70DC0822F90E02E3010F4C4
:1015A000089701C00E9791E001C0990F8A95EAF75C
:1015B000892F8D8B8C8D9D8D0197F1F7CE01DF9159
:1015C000CF910C9430090E9624E1FC0111922A95DA
:1015D000E9F70895CF93DF93EC01625F7F4F0E949C
:1015E0008B1ECE01DF91CF910895CF93DF93EC0155
:1015F0006E5E7F4F0E948B1ECE01DF91CF910895CA
:10160000CF93DF93EC016A5E7F4F0E948B1ECE0169
:10161000DF91CF910895CF93DF93EC01625E7F4F0E
:101620000E948B1ECE01DF91CF91089580E3FB01D4
:1016300080833296842F82958F7090E1899F401924
:1016400011244A3014F4405D01C0495C4293882360
:1016500011F0482FEFCF08950F9300E020E040E015
:1016600060E08DEF92E00E947F1E0F9108956F92CF
:101670007F928F929F92AF92BF92CF92DF92EF9222
:10168000FF920F931F93CF93DF93CDB7DEB7AC9745
:101690000FB6F894DEBF0FBECDBF7C01862EB42EF0
:1016A000A52E20E2922ECE0101966C01FC01292D7F
:1016B00011922A95E9F70FEF2FEF4FEF6FEF869614
:1016C0000E947F1E8EE992E09AA389A389A59AA51C
:1016D000ABA5BCA58BA39CA3ADA3BEA38701095B4F
:1016E0001F4F43E450E0BE016F5D7F4FC8010E9471
:1016F000E114019609F4BFC081E089838A8386E002
:10170000782E7B821C82F7016481758186819781A6
:101710000E94BE236D837E838F839887A986BA86B5
:1017200080E890E09C878B874CE150E0B601C801CF
:101730000E94ED14F601292D11922A95E9F757011F
:1017400088E0A80EB11CF501D60101900D927A94A3
:10175000E1F740E150E0B601C8010E94ED14F60146
:1017600011929A94E9F796E0692E712C40E250E0CC
:10177000B601C8010E94ED14F1E06F1A7108B1F7CB
:1017800083E6898392E89A8393E59B838C8385E340
:101790008D8381E08E838F829DE3988797E0998780
:1017A0008A8786E0F501DE011B9601900D928A95ED
:1017B000E1F78CE0898B8A8B6FE572E0CE0143966E
:1017C0000E94DC27F7014385BE01675E7F4FC7019A
:1017D0000E94160BF7014485BE01655E7F4FC7016D
:1017E0000E94160BF7014585BE01635E7F4FC7015E
:1017F0000E94160B4EE150E0B601C8010E94ED14A4
:10180000F3E08F121EC082E3898384E08A83F701AC
:1018100096859B8397859C8390899D8391899E83E0
:1018200096E39F838887828D8987838D8A87848DBD
:101830008B87858D8C874CE050E0B601C8010E94F3
:10184000ED1487E3898386E08A8391E09B8393E0AC
:101850009C838D838FE08E838AE38F838BE38887DD
:101860008FEF898749E050E0B601C8010E94ED146E
:10187000C8010E94E914AC960FB6F894DEBF0FBE03
:10188000CDBFDF91CF911F910F91FF90EF90DF902F
:10189000CF90BF90AF909F908F907F906F90089562
:1018A0002F923F924F925F926F927F928F929F9270
:1018B000AF92BF92CF92DF92EF92FF920F931F935E
:1018C000CF93DF93CDB7DEB7E3970FB6F894DEBFC3
:1018D0000FBECDBF7C012A013B0169010E94EC1AB9
:1018E0004B015C018701095B1F4FC8010E94601515
:1018F0001816190694F00E94EC1A681979098A09D9
:101900009B094616570668067906F0F062E370E018
:1019100080E090E00E941B1BE8CF42E250E0BE0155
:101920006F5F7F4FC8010E942A158981823031F490
:10193000F801858996898334910541F019A6C8017B
:101940000E94BA1489A566C18FEF64C16D817E8142
:101950008F8198850E94BE234B015C01F601608354
:1019600071838283938346E050E0B701685F7F4FC5
:10197000CE014D960E94B227892B99F4F701808100
:101980009181A281B38188169906AA06BB0648F008
:1019900084819581A681B78188159905AA05BB0523
:1019A00028F4C8010E94BA1480E034C189899A8958
:1019B000AB89BC89F70186879787A08BB18B3EECFA
:1019C000C32ED12CC8010E940115F1E0CF1AD10815
:1019D000C9F719A6C70182969BA78AA7F701B696F1
:1019E000FDA7ECA708969FA78EA73C976F018E9640
:1019F00099AB88AB3897FBABEAAB5701F6E1AF0E7A
:101A0000B11C47018EE1880E911CC8010E94A014F0
:101A1000181619060CF093CFC8010E9401158333E4
:101A2000910509F4CDC0F4F481309105B9F11CF4AD
:101A3000892B59F3DFC083309105C1F1069709F076
:101A4000D9C0C8010E9401153C0144E050E0B40136
:101A5000C8010E942A15212C312C7724F4E06F1A3A
:101A600071083FC08A33910509F47EC03CF4853388
:101A7000910561F0C69709F43FC0BCC08B33910556
:101A800009F488C08F3F910501F2B4C0C8010E94DB
:101A90000115C8010E94011589A7B7CFC8010E948E
:101AA000011544E050E06AA97BA93AC0C8010E9430
:101AB00001153C0144E050E0B501C8010E942A151F
:101AC000212C312C772494E0691A710826143704EC
:101AD0000CF09BCFC8010E940115EFEF2E1A3E0AB1
:101AE000F5CF261437040CF090CFC8010E940115E1
:101AF0008FEF281A380AF5CFC8010E940115782EF9
:101B0000F701828D811110C0838D81110DC0848DEC
:101B100081110AC0858D811107C044E050E0B601F3
:101B2000C8010E942A1571CFE8A9F9A92080318047
:101B300042805380B601CE0183960E948B1E8DA1F8
:101B40009EA1AFA1B8A582159305A405B50529F3FB
:101B5000212C312C721409F458CFC8010E940115B0
:101B6000FFEF2F1A3F0AF6CFC8010E94011544E08B
:101B700050E06CA57DA5C8010E942A15F70166A159
:101B800077A180A591A50E94BE2366A377A380A715
:101B900091A73BCFC8010E94011544E050E06EA51B
:101BA0007FA5C8010E942A15F70162A573A584A527
:101BB00095A50E94BE2362A773A784A795A725CFEA
:101BC000C8010E94011544E050E06AA57BA5C80148
:101BD0000E942A15F70162A173A184A195A10E9418
:101BE000BE2362A373A384A395A366A777A780AB44
:101BF00091AB0BCFC8010E940115382E612C712CBE
:101C0000361409F402CFC8010E940115FFEF6F1AC4
:101C10007F0AF6CFE3960FB6F894DEBF0FBECDBFB6
:101C2000DF91CF911F910F91FF90EF90DF90CF90B8
:101C3000BF90AF909F908F907F906F905F904F90EC
:101C40003F902F9008952F923F924F925F926F9204
:101C50007F928F929F92AF92BF92CF92DF92EF923C
:101C6000FF920F931F93CF93DF93CDB7DEB72797E4
:101C70000FB6F894DEBF0FBECDBF8C0120ED37E06C
:101C800040E050E061E070E080E090E00E942720BA
:101C9000D80114966D937D938D939C931797F801BB
:101CA00060837183828393834801F7E48F0E911CD4
:101CB000C4010E94CC1464E470E0C4010E94B11518
:101CC000882309F428C10E94EC1A6B017C01A12C25
:101CD000B12C1D82180186E4280E311CD801DE9635
:101CE000BF83AE8338EE432E33E0532E612C712C2C
:101CF000F1018081833009F4FDC081111FC0F8011A
:101D000084819581A681B7810196A11DB11D84832F
:101D10009583A683B7830E94EC1A6C197D098E09FE
:101D20009F09A30192010E947D23A90161E0C801DE
:101D30000E94370B81E0D1018C93BEC08430F9F44E
:101D4000F80184819581A681B7810196A11DB11DFD
:101D500084839583A683B7830E94EC1A6C197D094E
:101D60008E099F09A30192010E947D23A90163E0CE
:101D7000C8010E94370BE2E0D101EC939DC0813095
:101D800061F5AE81BF814D915D916D917C919E0118
:101D90002F5F3F4FC8010E94500C8D83823009F0A5
:101DA0008BC089819A81AB81BC81F8018483958342
:101DB000A683B7830E94EC1A6C197D098E099F09CE
:101DC000A30192010E947D23A90163E0C8010E9442
:101DD000370BED81D101EC9375C0823009F06CC0F6
:101DE000AE81BF814D915D916D917C919E012F5F80
:101DF0003F4FC8010E94500C8D83853009F056C0BA
:101E000083E0F1018083F80182A193A1A4A1B5A18F
:101E1000892B8A2B8B2B41F484E893E0A0E0B0E07F
:101E200082A393A3A4A3B5A3F80186A197A1A0A51B
:101E3000B1A5892B8A2B8B2B61F482A193A1A4A13C
:101E4000B5A1B695A7959795879586A397A3A0A7C3
:101E5000B1A7D8019A964D915D916D917C919D9716
:101E600096968D919D910D90BC91A02D452B462B62
:101E7000472B59F4AC01BD01440F551F661F771F56
:101E8000F80142A753A764A775A7F80186A797A7EB
:101E9000A0ABB1AB82A593A5A4A5B5A582AB93AB2E
:101EA000A4ABB5ABAA24A394B12C0CC0FD81F63031
:101EB00019F4D1011C9206C0BD81BF3F19F4F10194
:101EC00010821D82F1E0AF16B10409F411CF0E9417
:101ED000EC1A6C197D098E099F09D801DA962D91AB
:101EE0003D914D915C91DD972617370748075907BB
:101EF00008F0FECEC4010E94CC14F80184819581C3
:101F0000A681B7810196A11DB11D84839583A68307
:101F1000B783C50102C080E090E027960FB6F89421
:101F2000DEBF0FBECDBFDF91CF911F910F91FF900C
:101F3000EF90DF90CF90BF90AF909F908F907F9069
:101F40006F905F904F903F902F900895CF92DF92C7
:101F5000EF92FF920F931F93CF93DF93EC016B01EE
:101F60001AA21BA21CA21DA21EA21FA218A619A67D
:101F70001AA61BA61CA61DA61EAA1FAA18AE19AE3D
:101F80002AAF3BAF4CAF5DAFFC01FE96E082F18221
:101F9000028313838C01085F1F4F86E0F8011192C2
:101FA0008A95E9F7CE010E94E30A86E0F601D8019E
:101FB00001900D928A95E1F7FE01EA5BFF4F1082D6
:101FC000CE01DF91CF911F910F91FF90EF90DF90A5
:101FD000CF900C94230EFB01428153816481758163
:101FE000FC014283538364837583178216820895AC
:101FF000CF93FB0181918111FDCFFB0180E090E047
:1020000020E030E0CAE06191662309F12430310517
:1020100064F56E3271F48F3F910509F034F5DA0101
:10202000A20FB31F12968C932F5F3F4F80E090E07A
:10203000EACFDC01CA9FC001CB9F900D1124772706
:1020400067FD709560537109860F971FDCCF8F3F36
:10205000910509F054F4243031053CF4FA01E20F03
:10206000F31F828381E090E002C080E090E0CF9196
:1020700008950F9300E020E040E060E083E093E00B
:102080000E947F1E0F910895AF92BF92CF92DF9270
:10209000EF92FF920F931F93CF93DF9300D01F9285
:1020A000CDB7DEB76C017B010E94EC1AF601778395
:1020B00066838601085F1F4FB6016A5F7F4F42E06B
:1020C00050E0C8010E94ED1481E090E09A8389837A
:1020D00042E050E0BE016F5F7F4FC8010E94ED14E7
:1020E00080E091E09A83898342E050E0BE016F5F17
:1020F0007F4FC8010E94ED141A82198242E050E01D
:10210000BE016F5F7F4FC8010E94ED1442E050E0B6
:10211000BE016F5F7F4FC8010E94ED1442E050E0A6
:10212000BE016F5F7F4FC8010E94ED146701F60189
:102130008081882311F1F7016F018191811115C010
:102140005601AE18BF081A141B0494F4AB8241E088
:1021500050E0BE016D5F7F4FC8010E94ED14A501E4
:10216000B701C8010E94ED1403C08E3229F7E8CFF1
:102170007601FFEFEF1AFF0ADACF1B8241E050E051
:10218000BE016D5F7F4FC8010E94ED14E12CFF245A
:10219000F394FA82E98242E050E0BE016F5F7F4F24
:1021A000C8010E94ED14FA82E98242E050E0BE01CB
:1021B0006F5F7F4FC8010E94ED1481E090E00F90A7
:1021C0000F900F90DF91CF911F910F91FF90EF90A3
:1021D000DF90CF90BF90AF9008954F925F926F9233
:1021E0007F928F929F92AF92BF92CF92DF92EF92A7
:1021F000FF920F931F93CF93DF93CDB7DEB7639713
:102200000FB6F894DEBF0FBECDBF7C015B016A0143
:102210000E94EC1A2B013C018701085F1F4F45010A
:10222000A12CB12CC8010E9460151816190694F053
:102230000E94EC1A64197509860997098616970693
:10224000A806B906D0F062E370E080E090E00E945A
:102250001B1BE8CFF7014281538164817581818D19
:10226000928DA38DB48D481759076A077B0741F4F7
:10227000858D968DC59721F406C08FEF9FEFF9C02D
:102280008EEF9FEFF6C0C8010E94A0140C970CF4CB
:10229000EEC04CE050E0BE016F5F7F4FC8010E946E
:1022A0002A158B819C819827892798279A8B898B5F
:1022B000F7014681578129813A814217530711F46A
:1022C00097FD06C0C8010E94BA148CEF9FEFD1C0E1
:1022D0008F709270892B31F0C8010E94BA148BEF75
:1022E0009FEFC7C0AF80B884BA24AB24BA24A1142E
:1022F000B10419F0E12CF12C23C0C8010E94BA14DA
:102300008AEF9FEFB6C041E050E0BE01635F7F4FB0
:10231000C8010E942A158D8581111BC08D858111F0
:10232000F2CFC8010E940115C8010E940115C80121
:102330000E940115C8010E940115FFEFEF1AFF0A64
:102340008D819E81982789279827E816F906D8F26B
:102350000AC08D859FEF980F9D878823F9F2C801E9
:102360000E940115F6CFE12CF12C41E050E0BE01B6
:102370006D5E7F4FC8010E942A158B89982F907C33
:1023800061F4882371F08B899FEF980F9B8B8823D2
:1023900041F0C8010E940115F6CFC8010E94011545
:1023A0001B8A8B898111E1CF42E050E0BE01615F61
:1023B0007F4FC8010E942A1542E050E0BE01635FD2
:1023C0007F4FC8010E942A15C8010E940115C8014B
:1023D0000E940115C8010E940115C8010E94011543
:1023E00042E050E0BE016F5E7F4FC8010E942A1597
:1023F0008F8598898115914029F48D859E85811559
:10240000914019F0812C912C16C089899A898115E7
:10241000944031F0C8010E94BA1487EF9FEF29C0A1
:10242000B6016E5F7F4F44E050E0C8010E942A155C
:1024300081E090E01EC089899A899827892798278A
:102440008816990638F4C8010E9401152FEF821AE8
:10245000920AF1CF8FEFE81AF80AEA14FB0409F0A8
:1024600084CFC8010E94BA1486EF9FEF02C08DEF9F
:102470009FEF63960FB6F894DEBF0FBECDBFDF911E
:10248000CF911F910F91FF90EF90DF90CF90BF9071
:10249000AF909F908F907F906F905F904F90089536
:1024A0008F929F92AF92BF92CF92DF92EF92FF9264
:1024B0000F931F93CF93DF9300D000D000D0CDB700
:1024C000DEB78C015B016A010E94F80F4C01009796
:1024D00009F05DC0F801428153816481758180916A
:1024E000050390910603A0910703B09108034817D4
:1024F00059076A077B0709F44EC00E94EC1A78015D
:10250000F8E0EF0EF11C6F7077277C5FC7010E9427
:10251000B115813009F043C08EE992E09A83898336
:10252000F80182819381A481B5818B839C83AD83E3
:10253000BE8345E350E0BE016F5F7F4FC7010E943D
:10254000E114892B19F4812C912C1DC0B501C8010F
:102550000E944410892BB9F3C7010E94E914892B0A
:1025600091F333E0A32EB12CA60168E873E1C80112
:102570000E94ED104C01F1E0AF1AB10821F08F3F3D
:102580002FEF920789F3C7010E94CC1408C088245A
:102590008394912C04C09EEF892E99249A94C401AF
:1025A00026960FB6F894DEBF0FBECDBFDF91CF9158
:1025B0001F910F91FF90EF90DF90CF90BF90AF9061
:1025C0009F908F90089524E030E0AC0164E081E0BA
:1025D00090E00C941F1824E030E0AC0164E085E04A
:1025E00090E00C941F1826E030E0AC0164E089E034
:1025F00090E00C941F1824E030E0AC0164E08FE020
:1026000090E00C941F18AF92BF92CF92DF92EF929E
:10261000FF920F931F93CF93DF9300D000D000D091
:10262000CDB7DEB76C015B0182E690E00E94C51E6B
:102630008C0182E6F80111928A95E9F7C801895B5D
:102640009F4F0E94E415F6011783068381E493E00F
:102650000E94FC17C5010E94F31200E020E040E058
:1026600060E0CE0101960E947F1ECE0103960E947B
:10267000FB1218E8E12E13E1F12E00E010E020E655
:102680003AEE40E050E0B501F601868197810E9464
:10269000A60F8C018130910589F5F601668177815D
:1026A000CE0101960E94EA0ACE0103960E94FB1217
:1026B000F60166817781CE0101960E94000BCE0162
:1026C00003960E94E312F60166817781CE0101969E
:1026D0000E94F50ACE0103960E94EB12F601668174
:1026E0007781CE0101960E940B0B4B815C816D813D
:1026F0007E81F6014283538364837583C8012696E5
:102700000FB6F894DEBF0FBECDBFDF91CF911F9102
:102710000F91FF90EF90DF90CF90BF90AF90089512
:102720008F929F92AF92BF92CF92DF92EF92FF92E1
:102730000F931F93CF93DF93EC015B014A01690173
:1027400081E493E00E94FC17C5010E94F312C401CA
:1027500002960E94FB12C80102960E94E312C70172
:1027600002960E94EB12F6014281538164817581C9
:102770004A835B836C837D83DF91CF911F910F919F
:10278000FF90EF90DF90CF90BF90AF909F908F9091
:1027900008956F927F928F929F92AF92BF92CF9245
:1027A000DF92EF92FF920F931F93CF93DF93CDB7FA
:1027B000DEB76E970FB6F894DEBF0FBECDBF6C01CB
:1027C0005B017A014901380100E02FEF4FEF6FEF15
:1027D000CE0149960E947F1E2EE932E03A8329837A
:1027E0008B8D9C8DAD8DBE8D8B839C83AD83BE8385
:1027F00038872F83F30182819381A481B5818987F2
:102800009A87AB87BC873E872D87F40182819381AD
:10281000A481B5818F87988BA98BBA8B3C8B2B8B2E
:10282000F70142815381648175814D8B5E8B6F8B83
:10283000788FCE0101967C018E01095F1F4F9E01AA
:10284000235F3F4FAE014D5E5F4FB501C6010E9451
:1028500090136E960FB6F894DEBF0FBECDBFDF911A
:10286000CF911F910F91FF90EF90DF90CF90BF908D
:10287000AF909F908F907F906F900895CF93DF934C
:10288000EC010E94751EAE014E5F5F4F24E030E008
:1028900060E08FE090E00E942719CE01DF91CF9198
:1028A00008952EE932E0FC0131832083FB0142814F
:1028B000538164817581FC014283538364837583F2
:1028C00008950F9300E020E040E060E081E293E0B3
:1028D0000E947F1E89E093E00F910C94751E0F9368
:1028E00000E020E040E060E087E293E00E947F1E8D
:1028F0000F9108950F9300E020E040E060E08DE24A
:1029000093E00E947F1E0F910895DC01ED91FC91F0
:10291000008CF18DE02D09942EE932E0FC01318329
:102920002083FB014189528963897489FC014283B8
:102930005383648375830895FC018589968908957E
:10294000FC01818D928D0895CF93DF931F92CDB7B7
:10295000DEB76983DC01ED91FC910280F381E02D0B
:1029600041E050E0BE016F5F7F4F09950F90DF910E
:10297000CF910895CF93DF93EC01898D9A8D892BA8
:1029800041F0E881F9810680F781E02DCE010995BB
:10299000F4CFDF91CF910895CF93DF93EC018C8535
:1029A000883061F00E94B616EC85F0E0EE0FFF1F54
:1029B000EF5EFC4F1182108288E08C87DF91CF910F
:1029C0000895FC01108E178A6E5F7F4F84850C94EA
:1029D0008417FC0184850C94A917CF93DF93EC0135
:1029E0009A018F89988DAB01BC018C850E94561786
:1029F0002F89388D280F391F388F2F8BDF91CF917A
:102A000008950F931F93CF93DF931F92CDB7DEB737
:102A10008C01FC01818D928D892B59F041E050E0B1
:102A2000BE016F5F7F4F84850E9404171816190638
:102A30001CF08FEF9FEF08C0F801818D928D0197F8
:102A4000928F818F898190E00F90DF91CF911F91BC
:102A50000F910895CF93DF93EC01898D9A8D0097A4
:102A600019F48FEF9FEF10C04817590708F0AC0119
:102A70008C850E940417181619069CF7298D3A8D2B
:102A8000281B390B3A8F298FDF91CF910895CF936F
:102A9000DF931F92CDB7DEB7FC01218D328D232B42
:102AA00049F0BE016F5F7F4F84850E94481789817E
:102AB00090E002C08FEF9FEF0F90DF91CF910895CC
:102AC0000F931F93CF93DF93CDB7DEB728970FB641
:102AD000F894DEBF0FBECDBF8C01DC01ED91FC91FF
:102AE0000284F385E02D0995F801648581E493E083
:102AF0000E94CD18892B41F148E050E0BE016F5F84
:102B00007F4FD8011C968C910E9404171816190645
:102B1000ECF4BE016F5F7F4FC8010F960E949B1EB1
:102B20008D8190E0982F88272E81820F911DF801CA
:102B3000968B858B8F8190E0982F88272885820F30
:102B4000911D928F818F02C080E090E028960FB691
:102B5000F894DEBF0FBECDBFDF91CF911F910F91D3
:102B60000895FF920F931F93CF93DF93EC018B0196
:102B70008C85883011F5F12C6F2D6295660F607E83
:102B8000685F83E090E00E945D18811102C0FC86BE
:102B900006C08831E1F3F39488E0F812EDCF8C851C
:102BA000883059F01E870D871A8E198E20E0A801F3
:102BB00062E00E94C41681E001C080E0DF91CF9105
:102BC0001F910F91FF900895FC011382128248EE2D
:102BD00053E060E070E044835583668377838AE640
:102BE00092E09183808388E08487CF010F960C94D4
:102BF000751ECF92DF92EF92FF920F931F93CF93A8
:102C0000DF93CDB7DEB7AF970FB6F894DEBF0FBE38
:102C1000CDBF7C018B016A01CE0101960E94751E19
:102C2000CE0109960E94E415CE018A960E94751E77
:102C300069E073E0CE0184960E945114BE016C5D80
:102C40007F4FCE0101960E94EB0FAE01465D5F4FB4
:102C5000B801CE0101960E94501281309105C1F455
:102C6000D701ED91FC910088F189E02D8EE992E089
:102C70009DA38CA30CA51DA52EA53FA50EA31FA348
:102C800028A739A7A601BE016C5D7F4FC701099532
:102C9000AF960FB6F894DEBF0FBECDBFDF91CF91D8
:102CA0001F910F91FF90EF90DF90CF9008950F93B9
:102CB00000E020E040E060E083E393E00E947F1EBC
:102CC0000F9108950F9300E020E040E060E089E379
:102CD00093E00E947F1E0F910895AB01682F6295CB
:102CE000660F607E645F24E030E08CE090E00C943E
:102CF0001F189B01682F6295660F607E685FC9018F
:102D00000C945D1862E070E00C9479169B01682FBA
:102D10006295660F607E645FC9010C94D617CF93ED
:102D2000DF93C82FD62F472F64E070E00E948616ED
:102D30004D2F65E070E08C2FDF91CF910C948616BB
:102D4000462F62E070E00C948616CF93DF93C82F75
:102D5000D62F472F60E170E00E9486164D2F61E16B
:102D600070E08C2FDF91CF910C948616CF93C82FF3
:102D700040E150E0682F81E493E00E94D0196FEFAA
:102D80008C2FCF910C94A016EF92FF921F93CF93AC
:102D9000DF9300D0CDB7DEB7182F7A018FEF860F03
:102DA000853048F5812F2A8369830E94B6162A81CF
:102DB0006981462F422B60E070E0812F0E948616C9
:102DC000E114F10411F0B7010AC060913F03709162
:102DD00040036F5F7F4F7093400360933F03812FE9
:102DE0000E948F1641E050E0612F81E493E00E9441
:102DF000D01981E001C080E00F900F90DF91CF915A
:102E00001F91FF90EF900895DF92EF92FF920F9342
:102E10001F93CF93DF93D82E7B018A01682F81E423
:102E200093E00E94CD18EC01009799F463E070E004
:102E30008D2D0E947916843111F1882301F1C1E0B2
:102E4000D0E08C3111F4C0E0D0E0D195C195D1092A
:102E500016C0081719070CF4E8011C161D067CF4AF
:102E600000E09E01A7016D2D81E493E00E947F198F
:102E700040E450E06D2D81E493E00E94D019CE0132
:102E8000DF91CF911F910F91FF90EF90DF90089508
:102E90000F93AB0101E021E030E0682F81E493E083
:102EA0000E947F1981E090E00F910895BF92CF9228
:102EB000DF92EF92FF920F931F93CF93DF93B82E81
:102EC0007B016A01E901682F81E493E00E94981870
:102ED0008C179D0730F46B2D81E493E00E949818C5
:102EE000EC018E019601A7016B2D81E493E00E9415
:102EF000E918CE01DF91CF911F910F91FF90EF90D4
:102F0000DF90CF90BF9008951F93CF93DF93182F3A
:102F1000FB01EA018081811109C08181811106C014
:102F20008281811103C08381882369F0209759F041
:102F3000BF01812F0E946D16BE01812F0E94A51630
:102F400081E090E002C080E090E0DF91CF911F919E
:102F50000895CF93C82F40E250E0682F81E493E0BA
:102F60000E94D0198C2F0E94821684FD0CC08C2FD9
:102F70000E94821683FFF6CF68E18C2F0E94A01674
:102F800080E090E006C060E18C2F0E94A01681E0F6
:102F900090E0CF9108958EBD00000DB407FEFDCFE7
:102FA0008EB508952A9808952A9A08951F93CF936D
:102FB000DF9300D01F92CDB7DEB7182F4B836A8303
:102FC00099830E94D2179981892F0E94CB17812F54
:102FD0000E94CB176A81862F0E94CB174B81842FCA
:102FE0000E94CB170E94D41781E00F900F900F9092
:102FF000DF91CF911F910895CF93DF9368EE73E037
:1030000080E090E00E941B1B229A0E944008C0E0D2
:10301000DC2FD295DD0FD07ED45F42E06D2F8EE1A4
:1030200090E00E94D61742E06D2F8FE190E00E9461
:10303000D617CF5FC83061F7DF91CF910895CF9257
:10304000DF92EF92FF920F931F93CF93DF9300D005
:1030500000D0CDB7DEB7F82E89014B835C836A833D
:1030600099830E94D21789810E94CB178F2D0E94CD
:10307000CB176A81862F0E94CB174B81C42E5C81AF
:10308000D52E7601E00EF11ECE14DF0431F0F601EC
:1030900081916F010E94CB17F7CF0E94D417C8010E
:1030A0000F900F900F900F90DF91CF911F910F9184
:1030B000FF90EF90DF90CF9008951F93CF93DF9311
:1030C00000D0CDB7DEB7182F6A8399830E94D2173C
:1030D00089810E94CB17812F0E94CB176A81862F8E
:1030E0000E94CB1780E00E94CB1789830E94D417DF
:1030F00089810F900F90DF91CF911F9108951F93B9
:10310000CF93DF93182F60E270E00E947916C82FEA
:10311000D0E0DC2FCC2761E270E0812F0E9479168D
:103120009E01280F311DC901DF91CF911F91089594
:10313000FF920F931F93CF93DF93F62EC0E0D0E062
:103140008F2D0E947F188C01009721F08F2D0E94F7
:103150007F18EC01C017D10799F7CE01DF91CF910D
:103160001F910F91FF9008951F93CF93DF93182F16
:1031700066E270E00E947916C82FD0E0DC2FCC27E1
:1031800067E270E0812F0E9479169E01280F311DA1
:10319000C901DF91CF911F910895FF920F931F9363
:1031A000CF93DF93F62EC0E0D0E08F2D0E94B418AD
:1031B0008C01009721F08F2D0E94B418EC01C017EC
:1031C000D10799F7CE01DF91CF911F910F91FF9019
:1031D0000895CF92DF92EF92FF920F931F93CF93B8
:1031E000DF93D62EEA01790164E270E08D2D0E9412
:1031F0007916C82E65E270E08D2D0E947916C80FF1
:10320000D11D2C2D30E0322F2227C20FD31F6D2D60
:103210006295660F607E6C5E9801A701CE010E94E8
:103220001F18C00FD11F4D2F64E270E08D2D0E943A
:1032300086164C2F65E270E08D2DDF91CF911F91A6
:103240000F91FF90EF90DF90CF900C948616CF9265
:10325000DF92EF92FF920F931F93CF93DF9300D0F3
:1032600000D0CDB7DEB7F82E89014B835C836A832B
:1032700099830E94D21789810E94CB178F2D0E94BB
:10328000CB176A81862F0E94CB174B81C42E5C819D
:10329000D52E7601E00EF11ECE14DF0439F080E069
:1032A0000E94CB17F60181936F01F6CF0E94D417CD
:1032B000C8010F900F900F900F90DF91CF911F9149
:1032C0000F91FF90EF90DF90CF9008950F931F9391
:1032D000CF93DF9300D0CDB7DEB75A834983A901DE
:1032E000980189819A816295660F607E685E0F9071
:1032F0000F90DF91CF911F910F910C9427198F920E
:103300009F92AF92BF92CF92DF92EF92FF920F9374
:103310001F93CF93DF936C01962E5A017901802E73
:1033200068E270E0892D0E947916C82F69E270E08A
:10333000892D0E947916D0E0DC2FCC27C80FD11D33
:1033400087019501AE01692DC6010E9466198110A1
:103350001AC0CE0DDF1D4D2F68E270E0892D0E944E
:1033600086164C2F69E270E0892DDF91CF911F9175
:103370000F91FF90EF90DF90CF90BF90AF909F9014
:103380008F900C948616DF91CF911F910F91FF9033
:10339000EF90DF90CF90BF90AF909F908F90089567
:1033A000CF93C62F61E070E08C2F0E94861661E0FB
:1033B00070E08C2F0E9479168111F9CFCF9108957A
:1033C0000F931F9360934E0370934F0380935003AA
:1033D0009093510300910A0110910B0120910C016F
:1033E00030910D01060F171F281F391F0093460348
:1033F00010934703209348033093490382E090E001
:1034000090934503809344030E94EC1A60934A030F
:1034100070934B0380934C0390934D031F910F9136
:103420000895CF92DF92EF92FF920F931F930E9425
:10343000EC1AC0904A03D0904B03E0904C03F090FC
:103440004D036C197D098E099F0900914E0310915F
:103450004F032091500330915103683E7340810522
:103460009105D8F00F5F1F4F2F4F3F4F00934E0332
:1034700010934F03209350033093510348EEC40E32
:1034800043E0D41EE11CF11CC0924A03D0924B03CE
:10349000E0924C03F0924D03CACF80914603909185
:1034A0004703A0914803B0914903081719072A0759
:1034B0003B07C8F1E0914203F0914303309799F143
:1034C0000995611571058105910519F00E94E019B2
:1034D0002AC080910A0190910B01A0910C01B0913A
:1034E0000D0140914E0350914F0360915003709134
:1034F0005103840F951FA61FB71F80934603909317
:103500004703A0934803B093490381E090E02091E2
:10351000440330914503232B11F480E090E0909315
:1035200045038093440360914E0370914F03809153
:103530005003909151031F910F91FF90EF90DF90F6
:10354000CF9008951F920F920FB60F9211242F93D0
:103550003F938F939F93AF93BF9380915303909129
:103560005403A0915503B09156033091520323E0C8
:10357000230F2D3720F40196A11DB11D05C026E8AB
:10358000230F0296A11DB11D209352038093530374
:1035900090935403A0935503B0935603809157031F
:1035A00090915803A0915903B0915A030196A11D1F
:1035B000B11D8093570390935803A0935903B09380
:1035C0005A03BF91AF919F918F913F912F910F908F
:1035D0000FBE0F901F9018952FB7F894609153036A
:1035E0007091540380915503909156032FBF089515
:1035F0003FB7F8948091570390915803A0915903D5
:10360000B0915A0326B5A89B05C02F3F19F001962B
:10361000A11DB11D3FBF6627782F892F9A2F620FFA
:10362000711D811D911D42E0660F771F881F991F34
:103630004A95D1F708958F929F92AF92BF92CF9201
:10364000DF92EF92FF926B017C010E94F81A4B010E
:103650005C01C114D104E104F104F1F00E9458238B
:103660000E94F81A681979098A099B09683E734013
:103670008105910570F321E0C21AD108E108F10833
:1036800088EE880E83E0981EA11CB11CC114D104E1
:10369000E104F10429F7DDCFFF90EF90DF90CF90A8
:1036A000BF90AF909F908F900895789484B582607A
:1036B00084BD84B5816084BD85B5826085BD85B5D6
:1036C000816085BDEEE6F0E0808181608083E1E885
:1036D000F0E01082808182608083808181608083BD
:1036E000E0E8F0E0808181608083E1EBF0E08081C0
:1036F00084608083E0EBF0E0808181608083EAE792
:10370000F0E080818460808380818260808380811A
:10371000816080838081806880831092C1000895D9
:10372000833081F028F4813099F08230A1F008953F
:103730008730A9F08830B9F08430D1F480918000CE
:103740008F7D03C0809180008F77809380000895E3
:1037500084B58F7702C084B58F7D84BD0895809134
:10376000B0008F7703C08091B0008F7D8093B00050
:103770000895CF93DF9390E0FC01E458FF4F24912C
:10378000FC01E057FF4F8491882349F190E0880FB6
:10379000991FFC01E854FF4FA591B49182559F4FAA
:1037A000FC01C591D4919FB7611108C0F8948C9128
:1037B000209582238C93888182230AC0623051F441
:1037C000F8948C91322F309583238C938881822BAF
:1037D000888304C0F8948C91822B8C939FBFDF91D7
:1037E000CF9108950F931F93CF93DF931F92CDB77F
:1037F000DEB7282F30E0F901E859FF4F8491F90135
:10380000E458FF4F1491F901E057FF4F0491002352
:10381000C9F0882321F069830E94901B6981E02F01
:10382000F0E0EE0FFF1FE255FF4FA591B4919FB757
:10383000F8948C91611103C01095812301C0812BF4
:103840008C939FBF0F90DF91CF911F910F9108959F
:10385000CF93DF93282F30E0F901E859FF4F84918F
:10386000F901E458FF4FD491F901E057FF4FC4919B
:10387000CC2391F081110E94901BEC2FF0E0EE0F11
:10388000FF1FEC55FF4FA591B4912C912D2381E0A2
:1038900090E021F480E002C080E090E0DF91CF91E1
:1038A0000895FC01818D228D90E0805C9F4F821BEA
:1038B00091098F7399270895FC01918D828D981736
:1038C00031F0828DE80FF11D858D90E008958FEF26
:1038D0009FEF0895FC01918D828D981761F0828D84
:1038E000DF01A80FB11D5D968C91928D9F5F9F7334
:1038F000928F90E008958FEF9FEF08958EEE9DE1F7
:10390000892B49F080E090E0892B29F00E94EE1D80
:1039100081110C9400000895FC01848DDF01A80F33
:10392000B11DA35ABF4F2C91848D90E001968F73E7
:103930009927848FA689B7892C93A089B1898C9106
:1039400080648C93938D848D981306C00288F389CC
:10395000E02D80818F7D80830895CF93DF93EC01EC
:10396000888D8823C9F0EA89FB89808185FD05C09F
:10397000A889B9898C9186FD0FC00FB607FCF5CFD9
:10398000808185FFF2CFA889B9898C9185FFEDCF21
:10399000CE010E948C1CE7CFDF91CF910895CF928A
:1039A000DF92FF920F931F93CF93DF931F92CDB7B8
:1039B000DEB76C0181E0D60158968C9358975B96E0
:1039C0009C915B975C968C915C97981307C050967E
:1039D000ED91FC915197808185FD2EC0F601038DFC
:1039E00010E00F5F1F4F0F731127F02EF601848D2B
:1039F000F81211C00FB607FCF9CFD6015096ED9121
:103A0000FC915197808185FFF1CFC60169830E94A7
:103A10008C1C6981EBCF838DE80FF11DE35AFF4FBA
:103A20006083D6015B960C935B975296ED91FC9167
:103A30005397808180620CC0D6015696ED91FC911F
:103A4000579760835096ED91FC91519780818064E7
:103A5000808381E090E00F90DF91CF911F910F91D3
:103A6000FF90DF90CF900895BF92CF92DF92EF92B8
:103A7000FF92CF93DF93EC016A017B01B22EE889BC
:103A8000F98982E08083411581EE5807610571054F
:103A9000A1F060E079E08DE390E0A70196010E943B
:103AA0007D23215031094109510956954795379594
:103AB0002795211580E1380798F0E889F989108267
:103AC00060E874E88EE190E0A70196010E947D23F2
:103AD0002150310941095109569547953795279548
:103AE000EC85FD853083EE85FF852083188EEC897B
:103AF000FD89B082EA89FB89808180618083EA89BF
:103B0000FB89808188608083EA89FB898081806865
:103B10008083EA89FB8980818F7D8083DF91CF91CB
:103B2000FF90EF90DF90CF90BF9008951F920F927B
:103B30000FB60F9211242F938F939F93EF93FF93C0
:103B4000E0916B03F0916C038081E0917103F0913F
:103B5000720382FD12C09081809174038F5F8F7316
:103B600020917503821751F0E0917403F0E0E55A5B
:103B7000FC4F958F8093740301C08081FF91EF917A
:103B80009F918F912F910F900FBE0F901F901895BE
:103B90001F920F920FB60F9211242F933F934F93C2
:103BA0005F936F937F938F939F93AF93BF93EF93A5
:103BB000FF938BE593E00E948C1CFF91EF91BF91E6
:103BC000AF919F918F917F916F915F914F913F91B5
:103BD0002F910F900FBE0F901F9018958BE593E0DB
:103BE0000E94511C21E0892B09F420E0822F0895C6
:103BF00010925E0310925D0388EE93E0A0E0B0E0C7
:103C000080935F0390936003A0936103B09362037A
:103C10008EE892E090935C0380935B0385EC90E0E8
:103C2000909368038093670384EC90E090936A0319
:103C30008093690380EC90E090936C0380936B0316
:103C400081EC90E090936E0380936D0382EC90E0A2
:103C50009093700380936F0386EC90E090937203CF
:103C6000809371031092740310927503109276037F
:103C7000109277030895AF92BF92CF92DF92EF92A6
:103C8000FF920F931F93CF93DF936C017B01C0E0F2
:103C9000D0E000E010E0F601EC0FFD1F4AE050E03C
:103CA0006281C7010E94A01F5C016EE2C7010E94F1
:103CB000151F8A0D9B1D080F191F2196C330D105B2
:103CC00051F74AE050E0F6016581C7010E94A01F4C
:103CD000800F911FDF91CF911F910F91FF90EF9077
:103CE000DF90CF90BF90AF9008952EE932E0FC01B5
:103CF00031832083128213821482158208950F93D8
:103D0000FC018EE992E09183808362834383248364
:103D100005830F9108952EE932E0FC013183208361
:103D2000FB014081518162817381FC014283538395
:103D3000648375830895FB014081518162817381A1
:103D4000FC01428353836483758308958EE992E076
:103D50009093F9038093F8031092FA031092FB03F7
:103D60001092FC031092FD03089508950E94551BC4
:103D70000E94B51E0E940308CEE7DCE10E942F08D6
:103D80002097E1F30E947E1CF9CF0C940124CF927E
:103D9000DF92EF92FF920F931F93CF93DF937C01FB
:103DA0006A01EB0100E010E00C151D0571F069914E
:103DB000D701ED91FC910190F081E02DC7010995AB
:103DC000892B19F00F5F1F4FEFCFC801DF91CF9103
:103DD0001F910F91FF90EF90DF90CF9008956115A4
:103DE000710581F0DB010D900020E9F7AD01415034
:103DF0005109461B570BDC01ED91FC910280F381C8
:103E0000E02D099480E090E00895DC01ED91FC91B3
:103E1000DB0114964D915C9115976D917C91028018
:103E2000F381E02D09940C94EF1EDC01ED91FC91DF
:103E30000190F081E02D099460EA72E00C94EF1E8D
:103E40000F931F93CF93DF93EC010E94051F8C010A
:103E5000CE010E941C1F800F911FDF91CF911F91F7
:103E60000F9108950F931F93CF93DF93EC010E945E
:103E7000EF1E8C01CE010E941C1F800F911FDF914D
:103E8000CF911F910F9108958F929F92AF92BF9201
:103E9000DF92EF92FF920F931F93CF93DF93CDB7F3
:103EA000DEB7A1970FB6F894DEBF0FBECDBF7C0181
:103EB000F42FD52ECB0119A2223008F42AE08E016E
:103EC0000F5D1F4F822E912CA12CB12C6F2F7D2DB9
:103ED000A50194010E947D23F22FD32ECA01015027
:103EE00011096A3014F4E0E301C0E7E3E60FD801FA
:103EF000EC93232B242B252B49F7B801C7010E94F3
:103F0000EF1EA1960FB6F894DEBF0FBECDBFDF91B6
:103F1000CF911F910F91FF90EF90DF90BF90AF90E6
:103F20009F908F9008952115310541F4DC01ED91AA
:103F3000FC910190F081E02D642F09940C94441FB2
:103F40009A01462F50E060E070E00C94931F0F93AD
:103F50001F93CF93DF93EC010E94EC1A6887798757
:103F60008A879B87E881F9810680F781E02DCE0161
:103F7000099597FF15C00E94EC1A088519852A85B6
:103F80003B85601B710B820B930B0C811D812E8175
:103F90003F81601771078207930720F38FEF9FEF30
:103FA000DF91CF911F910F910895FC0144835583B8
:103FB000668377830895EF92FF920F931F93CF93B9
:103FC000DF93EC018B01E42E62EA72E00E94B120E3
:103FD000C8010E94A71FFF24E7FCF09497FD0BC0C7
:103FE0008E159F0541F0682FCE010E94FA21C8016D
:103FF0000E94A71FF3CFCE01DF91CF911F910F91A8
:10400000FF90EF900895CF93DF9300D000D0CDB70D
:10401000DEB79B01AC01611571058105910569F061
:1040200069833A834B835C830E94772529813A8197
:104030004B815C810E949F2303C060E070E0CB0154
:104040000F900F900F900F90DF91CF910895CF9226
:10405000DF92EF92FF926B017C0162177307840776
:10406000950764F4CA01B9016C197D098E099F098D
:104070000E9403206C0D7D1D8E1D9F1DFF90EF90F3
:10408000DF90CF900895FC01808191810C94992458
:10409000CF93DF93EC0188819981009711F00E9402
:1040A0009924198218821D821C821B821A82DF9138
:1040B000CF9108950F931F93CF93DF93EC018B0162
:1040C0006F5F7F4F888199810E948525009731F02D
:1040D000998388831B830A8381E001C080E0DF919C
:1040E000CF911F910F910895CF93DF93EC018881B9
:1040F0009981892B29F08A819B818617970760F423
:10410000CE010E945A20882341F08C819D81892B09
:1041100019F4E881F981108281E0DF91CF9108954F
:10412000EF92FF920F931F93CF93DF93EC017B01EC
:104130008A01BA010E947420811104C0CE010E943C
:10414000482007C01D830C83B701888199810E9494
:10415000DC27CE01DF91CF911F910F91FF90EF905F
:104160000895FC011182108213821282158214823A
:104170006115710559F0FB0101900020E9F7AF01CD
:1041800041505109461B570B0C94902008950F93F2
:104190001F93CF93DF938C01EB01FC018081918110
:1041A000009799F0428153812C813D81421753073A
:1041B00050F0688179810E94DC278C819D81F80113
:1041C0009583848313C00E94992488819981F80182
:1041D000918380838A819B81938382838C819D815B
:1041E00095838483198218821B821A821D821C8205
:1041F000DF91CF911F910F910895CF93DF93EC0141
:10420000FB018617970761F0608171816115710567
:1042100029F0448155810E94902002C00E944820CC
:10422000CE01DF91CF910895FC011182108213829B
:104230001282158214820C94FD20CF93DF93EC013F
:104240008617970711F00E94C720CE01DF91CF910A
:104250000895CF93DF93EC016115710561F0FB01C7
:1042600001900020E9F7AF0141505109461B570B5F
:104270000E94902002C00E944820CE01DF91CF9181
:1042800008950F931F93CF93DF93CDB7DEB7629757
:104290000FB6F894DEBF0FBECDBF8C01CB01F80185
:1042A00011821082138212821582148250E0BE01A4
:1042B0006F5F7F4F0E940C28BE016F5F7F4FC80168
:1042C0000E94292162960FB6F894DEBF0FBECDBFC3
:1042D000DF91CF911F910F9108950F931F93CF936B
:1042E000DF93CDB7DEB7A2970FB6F894DEBF0FBE4F
:1042F000CDBF8C01CB01BA01F8011182108213826B
:1043000012821582148230E0AE014F5F5F4F0E942F
:104310002228BE016F5F7F4FC8010E942921A2960B
:104320000FB6F894DEBF0FBECDBFDF91CF911F91C6
:104330000F9108950F931F93CF93DF93CDB7DEB7FF
:10434000A1970FB6F894DEBF0FBECDBF8C01CB0195
:10435000BA01F8011182108213821282158214822E
:1043600030E0AE014F5F5F4F0E945128BE016F5F8A
:104370007F4FC8010E942921A1960FB6F894DEBF95
:104380000FBECDBFDF91CF911F910F910895EF9296
:10439000FF920F931F93CF93DF93EC017B010C816E
:1043A0001D816115710511F480E016C0411551059C
:1043B00091F0040F151FB8010E9474208823A1F307
:1043C000288139818C819D81B701820F931F0E94C2
:1043D000DC271D830C8381E0DF91CF911F910F912A
:1043E000FF90EF900895FB014481558160817181B8
:1043F0000C94C721CF93DF9300D0CDB7DEB769838C
:104400001A8241E050E0BE016F5F7F4F0E94C721DA
:104410000F900F90DF91CF910895CF93DF93EC0130
:10442000FB0144815581608171810E94C721811106
:1044300003C0CE010E944820CE01DF91CF910895A4
:10444000FC0124813581232B31F421E061157105B4
:10445000A1F0FB0108C0FC0180819181611571050B
:1044600031F421E0FC018081882339F005C00E94ED
:10447000D32721E0892B09F020E0822F08950F93A4
:104480001F93CF93DF93EB0141155105E9F020977E
:10449000D9F0FC016481758126173707A0F4621BEF
:1044A000730B8A01015011096017710708F48B0121
:1044B000FC0160817181620F731FA801CE010E940F
:1044C000E327C00FD11F1882DF91CF911F910F9169
:1044D0000895CF93DF93FC01848195814817590794
:1044E00078F4C081D181772767FD7095CE01840F64
:1044F000951F0E94C827009719F08C1B9D0B02C0C6
:104500008FEF9FEFDF91CF91089540E050E00C9442
:104510006922CF93DF93FC01848195814817590765
:1045200078F4C081D181FB0160817181CE01840F5B
:10453000951F0E94F227009719F08C1B9D0B02C05B
:104540008FEF9FEFDF91CF91089540E050E00C9402
:104550008922BF92CF92DF92EF92FF920F931F9327
:10456000CF93DF936C017B01EA01890124173507A2
:1045700020F48D2FE901042F182F62EA72E0C601A2
:104580000E94B120D70114968D919C911597C81760
:10459000D907C8F48017910708F48C01D701ED9171
:1045A000FC911197E00FF11FB08010826D917C910A
:1045B0006C0F7D1FC6010E942921D701ED91FC914E
:1045C000E00FF11FB082C601DF91CF911F910F91D3
:1045D000FF90EF90DF90CF90BF900895AF92BF9281
:1045E000CF92DF92EF92FF920F931F93CF93DF93BF
:1045F0007C01DC01CD90DC901197C114D10409F449
:1046000041C01496CD91DC9115972097D9F15601B0
:104610008501BFEFAB1ABB0AF8018081992787FD9E
:1046200090950E94AA27892B99F72197CC0DDD1D23
:104630008881992787FD90950E94AA27892B91F45C
:10464000AE014F5F5F4F401B510BD70115965C9336
:104650004E931497C016D10650F4B801C6010E94BB
:10466000BF2705C0C017D10758F32197E1CFD70165
:10467000ED91FC91119714968D919C911597E80FEF
:10468000F91F1082DF91CF911F910F91FF90EF9052
:10469000DF90CF90BF90AF900895FC018081918111
:1046A000009711F00C94832760E070E0CB0108952F
:1046B0000895DB018F939F930E94D423BF91AF9104
:1046C000A29F800D911DA39F900DB29F900D11246C
:1046D000089597FB072E16F4009407D077FD09D0B4
:1046E0000E94E72307FC05D03EF4909581959F4FEB
:1046F0000895709561957F4F0895A1E21A2EAA1B27
:10470000BB1BFD010DC0AA1FBB1FEE1FFF1FA21781
:10471000B307E407F50720F0A21BB30BE40BF50B7E
:10472000661F771F881F991F1A9469F76095709507
:10473000809590959B01AC01BD01CF010895052E98
:1047400097FB1EF400940E94B62357FD07D00E94E9
:104750007D2307FC03D04EF40C94B623509540956E
:10476000309521953F4F4F4F5F4F0895909580951D
:10477000709561957F4F8F4F9F4F089569279627BA
:1047800069277827872778270895A29FB001B39FCC
:10479000C001A39F700D811D1124911DB29F700D4A
:1047A000811D1124911D08950E94C523A59F900D80
:1047B000B49F900DA49F800D911D11240895B7FF03
:1047C0000C94D4230E94D423821B930B0895AA1B1C
:1047D000BB1B51E107C0AA1FBB1FA617B70710F0EC
:1047E000A61BB70B881F991F5A95A9F7809590951E
:1047F000BC01CD010895EE0FFF1F0590F491E02D4F
:104800000994CF93DF938230910510F482E090E019
:10481000E0910004F091010420E030E0A0E0B0E07D
:10482000309739F14081518148175907B8F048173E
:10483000590771F482819381109729F013969C9304
:104840008E9312972CC0909301048093000427C08C
:104850002115310531F04217530718F0A901DB018A
:1048600001C0EF019A01BD01DF010280F381E02D5B
:10487000D7CF21153105F9F0281B390B243031052C
:1048800080F48A819B816115710521F0FB0193837E
:10489000828304C09093010480930004FE01329649
:1048A00044C0FE01E20FF31F81939193225031091E
:1048B000398328833AC02091FE033091FF03232BD4
:1048C00041F420910201309103013093FF032093C2
:1048D000FE0320910001309101012115310541F4C1
:1048E0002DB73EB74091040150910501241B350BB3
:1048F000E091FE03F091FF03E217F307A0F42E1BF3
:104900003F0B2817390778F0AC014E5F5F4F241733
:10491000350748F04E0F5F1F5093FF034093FE038F
:104920008193919302C0E0E0F0E0CF01DF91CF915D
:104930000895CF93DF93009709F487C0FC01329765
:1049400013821282C0910004D0910104209781F457
:1049500020813181280F391F8091FE039091FF0340
:104960008217930779F5F093FF03E093FE036DC080
:10497000DE0120E030E0AE17BF0750F412964D91F3
:104980005C9113979D014115510509F1DA01F3CFAF
:10499000B383A28340815181840F951F8A179B079F
:1049A00071F48D919C911197840F951F02969183BC
:1049B000808312968D919C91139793838283211506
:1049C000310529F4F0930104E09300043EC0D901BD
:1049D0001396FC93EE9312974D915D91A40FB51F22
:1049E000EA17FB0779F480819181840F951F029665
:1049F000D90111969C938E938281938113969C93F7
:104A00008E931297E0E0F0E08A819B81009719F085
:104A1000FE01EC01F9CFCE01029628813981820F87
:104A2000931F2091FE033091FF032817390769F483
:104A3000309729F4109201041092000402C01382EE
:104A40001282D093FF03C093FE03DF91CF910895AC
:104A50008F929F92AF92BF92CF92DF92EF92FF928E
:104A6000CF93DF93EC01688179818A819B81611505
:104A700071058105910521F464E279ED8BE597E0FC
:104A80002DE133EF41E050E00E949F2349015A019C
:104A90009B01AC01A7EAB1E40E94D4236B017C0125
:104AA000ACEEB4EFA50194010E94E223C60ED71E1E
:104AB000E81EF91EF7FE06C081E0C81AD108E10819
:104AC00080E8F80AC882D982EA82FB82C701B6016F
:104AD0009F77DF91CF91FF90EF90DF90CF90BF90C5
:104AE000AF909F908F9008950E942825089586E0AA
:104AF00091E00E94282508956093060170930701B4
:104B000080930801909309010895A0E0B0E0EBE8DC
:104B1000F5E20C94AF28EC01CB01209719F40E9428
:104B20000124B8C0FE01E60FF71F9E012250310993
:104B3000E217F30708F4ACC0D9010D911C9111974D
:104B400006171707B8F00530110508F49FC0A80133
:104B5000445051094617570708F498C002501109EC
:104B6000061B170B019311936D937C93CF010E9449
:104B700099248CC05B01A01AB10A4E01800E911ECF
:104B8000A0910004B0910104612C712C60E070E0F0
:104B9000109709F449C0A815B905C9F5ED90FC9026
:104BA0001197670142E0C40ED11CCA14DB0478F1EE
:104BB00047018A189B08640142E0C40ED11C12967A
:104BC000BC9012971396AC91B5E0CB16D10440F08F
:104BD000B282A38391828082D9018D939C9309C074
:104BE0000E5F1F4F0E0D1F1DF90111830083EB2D6A
:104BF000FA2F6115710531F0DB011396FC93EE93EA
:104C0000129744C0F0930104E09300043FC06D91FB
:104C10007C9111976616770608F43B01BD01129648
:104C20000D90BC91A02DB4CF6091FE037091FF0355
:104C300068157905E9F468167906D0F44091000109
:104C4000509101014115510541F44DB75EB7609196
:104C5000040170910501461B570BE417F507C0F4DA
:104C6000F093FF03E093FE03F901918380830EC06C
:104C70000E9401247C01009759F0A801BE010E9406
:104C8000BF27CE010E949924C70104C0CE0102C0F3
:104C900080E090E0CDB7DEB7EEE00C94CB282F9209
:104CA0003F925F926F927F928F929F92AF92BF924C
:104CB000CF92DF92EF92FF920F931F93CF93DF93E8
:104CC0008B01EA016115710521F0DB018C931196CE
:104CD0009C93209739F09E012250310923323105EF
:104CE00008F0FBC07C016701BFEFCB1ADB0A56015D
:104CF000F7016080862D90E00E94AA27892B11F091
:104D00007601F1CFFDE26F120AC0570182E0A80ED2
:104D1000B11CD70111966C90772473940BC0BBE241
:104D20006B1207C05701E2E0AE0EB11CD70111961D
:104D30006C90712CCE018F7E892B89F4B0E36B12BD
:104D400022C0F50180818F7D883541F56180F2E0D8
:104D5000AF0EB11C872D8260782EC0E1D0E0C83044
:104D6000D105F1F04CF4C230D10511F5C12CD12C94
:104D7000E12CB0E4FB2E2FC0CA30D10531F0C03198
:104D8000D10521F115C0209751F7CAE0D0E0ACEC75
:104D9000CA2EDC2CEC2CACE0FA2E1DC02097F9F6C4
:104DA000C8E0D0E0C12CD12CE12CF0E1FF2E13C0E3
:104DB00060E070E080E090E89E01442737FD409578
:104DC000542F0E947D2369017A0105C0C12CD12C8A
:104DD000E12CE8E0FE2EF50160E020E030E0A901E2
:104DE0004E01AA2497FCA094BA2C1F0170ED572EF7
:104DF000560CA9E0A51570F48FEB860D8A3118F4D6
:104E000099EC592E06C08FE9860D8A3130F589EA72
:104E1000582E560C852D90E08C179D07F4F467FDF5
:104E200018C0C216D306E406F50680F0C501B40129
:104E30000E9459239B01AC01250D311D411D511DBF
:104E4000213031054105B0E85B0710F06FEF01C07C
:104E500061E03196D1016C90C8CF872D817001152A
:104E6000110571F0662329F03197D801ED93FC9379
:104E700007C071FE19C03297D801ED93FC9314C09E
:104E800067FF12C0882329F020E030E040E050E8BE
:104E900004C02FEF3FEF4FEF5FE782E290E0909387
:104EA00003048093020416C0882341F05095409576
:104EB000309521953F4F4F4F5F4F0CC057FF0AC0B1
:104EC00082E290E090930304809302042FEF3FEF7F
:104ED0004FEF5FE7B901CA0104C060E070E080E015
:104EE00090E0DF91CF911F910F91FF90EF90DF90B5
:104EF000CF90BF90AF909F908F907F906F905F907A
:104F00003F902F9008951F93FC0199278827BC019B
:104F1000E89411911032E9F3193010F01E30C8F303
:104F20001B3251F01D3249F4689406C00E943C289F
:104F3000610F711D811D911D119110531A30B0F335
:104F40003EF490958095709561957F4F8F4F9F4F60
:104F50001F9108959111ECC0803219F0895085504D
:104F6000D0F70895FB01DC0104C08D9101908019F8
:104F700021F441505040C8F7881B990B0895FB015C
:104F8000DC0102C001900D9241505040D8F70895C5
:104F9000FC018191861721F08823D9F7992708957C
:104FA0003197CF010895FB01DC018D9101908019AB
:104FB0000110D9F3990B0895FB01DC0101900D92CA
:104FC0000020E1F70895FB01DC014150504048F01A
:104FD00001900D920020C9F701C01D924150504030
:104FE000E0F70895FB0151915523A9F0BF01DC01C1
:104FF0004D9145174111E1F759F4CD010190002081
:1050000049F04D9140154111C9F3FB014111EFCF1A
:1050100081E090E0019708954532510520F4423037
:1050200010F00C941728FB011082CB010895BB27C8
:105030004A3031F4992322F4BDE2909581959F4F37
:105040000C947F282532310520F4223010F00C9486
:105050002D28FA011082CA010895BB272A3051F485
:10506000992342F4BDE290958095709561957F4FAC
:105070008F4F9F4F0C945D28592F482F372F262F85
:10508000660F771F881F991F660F771F881F991F4C
:10509000620F731F841F951F660F771F881F991F4C
:1050A00008952532310520F4223010F00C945C284C
:1050B000FA011082CA010895BB27FA01A62F6217D0
:1050C000710581059105330B30FB66F0AA27660F49
:1050D000771F881F991FAA1FA21710F0A21B6395A4
:1050E0003850A9F7A05DAA3308F0A95DA19336F75F
:1050F000B111B1931082CA010C949B28BB27FB010C
:105100005527AA27880F991FAA1FA41710F0A41BC0
:1051100083955051B9F7A05DAA3308F0A95DA1931A
:10512000009779F7B111B1931192CB010C949B28A0
:10513000992788270895DC01FC01672F7191772357
:10514000E1F7329704C07C916D9370836291AE1742
:10515000BF07C8F308952F923F924F925F926F92CC
:105160007F928F929F92AF92BF92CF92DF92EF92F7
:10517000FF920F931F93CF93DF93CDB7DEB7CA1B78
:10518000DB0B0FB6F894DEBF0FBECDBF09942A88A3
:10519000398848885F846E847D848C849B84AA844B
:1051A000B984C884DF80EE80FD800C811B81AA81D8
:1051B000B981CE0FD11D0FB6F894DEBF0FBECDBFA3
:0851C000ED010895F894FFCF02
:1051C800000004048000010000002C01000090A2EF
:1051D800DA104FA4642D3E3A200053746172742093
:1051E8004E6574776F726B210044484350205265B6
:1051F80071756573740044484350204661696C6555
:10520800642C20557365204C696E6B2D4C6F63615F
:105218006C204164726573730045746865726E65CD
:10522800742053746172746564212049503A2000D7
:1052380030413030364142374145373900496E698F
:10524800742E2E2E2E00743D007461670074616701
:105258003D003B74696D653D003B6A6F623D003BF4
:105268006F6E6C696E653D006A6F62006F6E6C6987
:105278006E650074696D65007365744A6F620073CA
:1052880065744F6E6C696E65006B6565700068616A
:1052980073436F756E74006461746153746F7265E3
:1052A8000067657453746F726500693C2D3A20007D
:1052B800726571756573744B6565703D310067651E
:1052C800744A6F623D31006765744F6E6C696E6534
:1052D8003D310067657453746F7265436F756E7402
:1052E8003D310067657453746F7265446174613D44
:1052F8003100496E6974206C6F6164696E672100C2
:10530800496E69742066696E697368656421000076
:105318000000009708C71E02097608EA08E908573E
:10532800495A6E65740000000000A414ED14A0141E
:1053380001154715BA14B115CC14E114F915E9147F
:1053480060152A1585148C149C1400000000CF1CCD
:10535800C71E511C6A1C5C1CAD1C000000003B1ED3
:105368000D0A006E616E00696E66006F7666000059
:00000001FF
